:10000000B2C00000CBC00000C9C00000C7C00000E3
:10001000C5C00000C3C00000C1C00000BFC00000D8
:10002000BDC00000BBC00000AAC30000B7C00000F4
:10003000B5C00000B3C00000B1C00000AFC00000F8
:10004000ADC00000ABC00000A9C00000A7C0000008
:10005000A5C00000A3C00000A1C000009FC0000018
:100060009DC000009BC0000099C0000097C0000028
:1000700095C0000093C0000091C000008FC0000038
:100080008DC000008BC0000089C0000087C0000048
:1000900085C0000083C0000081C000007FC0000058
:1000A0007DC000007BC0000079C000001A034C0036
:1000B00055004600410020004300480041004E002A
:1000C00047004500440000002A0344006500610029
:1000D0006E002000430061006D0065005200410089
:1000E00020004300480041004E0047004500440006
:1000F000200000000403090409022200010100C0DD
:10010000320904000001030000000921110100016F
:10011000223A0007058103080005120110010000C2
:100120000008EB034320010001020001050109045E
:10013000A1010901A100093009310932169CFF26ED
:10014000640036FFFF460100950375088102C00573
:100150000919012902150025017501950281027511
:100160000695018101C011241FBECFEFDAE0DEBF8A
:10017000CDBF11E0A0E0B1E0EEE3F0E102C00590F8
:100180000D92A031B107D9F721E0A0E1B1E001C0A3
:100190001D92A132B207E1F71AD04FC731CF84B711
:1001A000877F84BF0FB6F894A8958091600088611E
:1001B00080936000109260000FBE90E080E80FB660
:1001C000F89480936100909361000FBEBBC2E7DF9B
:1001D000789480E091E05BD6FAD4FBCF089508953F
:1001E00080E091E041D6E2EEF0E08081846080839F
:1001F000089580E091E005C580910E0190910F0176
:10020000009729F0019790930F0180930E010895B4
:100210000F931F9384E090E0F8019183808380E046
:100220001F910F9108950895292F33272330310509
:10023000E1F058F42130310599F02230310569F5AB
:1002400082E290E028EF30E02CC02132310501F14C
:100250002232310511F58AE390E02CE231E021C031
:1002600082E190E02AE131E01CC0992781309105BC
:1002700049F028F0029789F4ECEAF0E005C0E4EFD9
:10028000F0E002C0E8ECF0E0849190E09F0109C04A
:1002900089E090E02AE031E004C080E090E020E0D6
:1002A00030E0FA01318320830895CF92DF92EF92FC
:1002B000FF920F931F93CF93DF93EC018B017A0191
:1002C000CED1811133C0E114F10439F0F7018081FE
:1002D0009181081B190BC80FD91FC12CD12C0115F6
:1002E000110519F18091E80085FD16C08091E800A4
:1002F0008E778093E8006BD4E114F10449F0F701A4
:1003000080819181C80ED91ED182C08285E00EC045
:10031000A6D1882321F30AC089918093F10001506E
:100320001109FFEFCF1ADF0ADACF80E0DF91CF911A
:100330001F910F91FF90EF90DF90CF900895209143
:100340001F01309120012617370748F0611571050C
:1003500039F42091E8002E772093E80001C0B9011C
:10036000FC0120E06115710579F180911801882365
:10037000F1F18530F1F18091E80083FD3CC080917E
:10038000E80082FD2EC08091E80080FFEBCF209135
:10039000F3008091F20090E0922B6115710551F00D
:1003A0008830910538F421912093F1006150710952
:1003B0000196F3CF21E0089709F020E08091E80052
:1003C0008E778093E800CECF2111CFCF0AC08091E5
:1003D0001801882361F0853061F08091E80083FD89
:1003E0000AC08091E80082FFF2CF80E0089582E0A9
:1003F000089583E0089581E008956115710529F459
:100400002091E8002B772093E800FC01611571052D
:1004100041F180911801882361F1853061F180916B
:10042000E80083FD24C08091E80082FFEFCF209197
:10043000F3008091F20090E0922B892B31F08091B3
:10044000F10081936150710991F78091E8008B77F9
:100450008093E800DBCF80911801882351F085302C
:1004600051F08091E80080FFF6CF80E0089581E0B0
:10047000089582E0089583E0089520911F0130914E
:1004800020012617370748F06115710539F42091CE
:10049000E8002E772093E80001C0B901FC0120E0BC
:1004A0006115710591F180911801882309F440C00C
:1004B000853009F43FC08091E80083FD3DC0809104
:1004C000E80082FD2FC08091E80080FFE9CF2091F5
:1004D000F3008091F20090E0922B6115710559F0C4
:1004E0008830910540F424912093F10031966150B9
:1004F00071090196F2CF21E0089709F020E0809180
:10050000E8008E778093E800CBCF2111CCCF0AC0D2
:1005100080911801882361F0853061F08091E800B6
:1005200083FD0AC08091E80082FFF2CF80E0089549
:1005300082E0089583E0089581E00895982F973030
:1005400068F59093E900981739F07091EC002091CC
:10055000ED005091F00003C0242F762F50E021FDD4
:1005600002C09F5FECCF3091EB003E7F3093EB00F9
:100570003091ED003D7F3093ED003091EB00316024
:100580003093EB007093EC002093ED005093F0005B
:100590002091EE0027FDE5CF80E008958F708093D5
:1005A000E90081E008950F931F93CF93DF93062F07
:1005B000EC0110E0101771F16881611103C01F5F39
:1005C0002596F8CF2C81A981BA819B81862F8F70C7
:1005D000873010F080E01FC0223010F442E001C0EC
:1005E00046E0E8E0F0E020E0EA17FB0720F42F5FA8
:1005F000EE0FFF1FF9CF2295207F422B50E4959FED
:1006000090011124661F6627661F622B97DF8111F8
:10061000D6CFE0CF81E0DF91CF911F910F91089568
:100620008091190187FF11C08091E80082FD05C00B
:10063000809118018111F8CF11C08091E8008B776B
:100640000BC080911801882349F08091E80080FF59
:10065000F8CF8091E8008E778093E800089520918C
:10066000E4003091E50095E64091EC00842F817024
:1006700040FF23C08091E80080FD1DC080911801DB
:10068000882399F0853099F08091EB0085FD11C0A9
:100690004091E4005091E5002417350729F391506B
:1006A00011F09A01E1CF84E0089582E0089583E09B
:1006B000089581E0089580E008954091E80042FFA8
:1006C000DDCF08950F931F93CF93DF934BD052D07C
:1006D000C8EDD0E088818F7788838881806888839F
:1006E00088818F7D888319BC1092180110921401A3
:1006F000109216011092150100EE10E0F8018081B1
:100700008B7F808388818160888342E060E080E025
:1007100015DFE1EEF0E080818E7F8083E2EEF0E095
:10072000808181608083808188608083F8018081FE
:100730008E7F8083888180618883DF91CF911F9134
:100740000F910895E8EDF0E080818F7E8083E7EDE2
:10075000F0E080818160808384E082BF81E08093CB
:100760001701B0CFE8EDF0E080818E7F808310929A
:10077000E20008951092DA001092E10008951F92AD
:100780000F920FB60F9211242F933F934F935F93C5
:100790006F937F938F939F93AF93BF93EF93FF9349
:1007A0008091E10082FF0AC08091E20082FF06C0D2
:1007B0008091E1008B7F8093E1001EDD8091DA0063
:1007C00080FF1DC08091D80080FF19C08091DA00A1
:1007D0008E7F8093DA008091D90080FF0CC080E189
:1007E00089BD82E189BD09B400FEFDCF81E080931F
:1007F0001801F4DC04C019BC10921801F0DC8091DF
:10080000E10080FF18C08091E20080FF14C0809159
:10081000E2008E7F8093E2008091E200806180930D
:10082000E2008091D80080628093D80019BC85E0F6
:1008300080931801CBD18091E10084FF2FC080917B
:10084000E20084FF2BC080E189BD82E189BD09B44B
:1008500000FEFDCF8091D8008F7D8093D8008091DD
:10086000E1008F7E8093E1008091E2008F7E809393
:10087000E2008091E20081608093E20080911401A7
:10088000882311F084E007C08091E30087FD02C057
:1008900081E001C083E08093180198D18091E1004C
:1008A00083FF22C08091E20083FF1EC08091E1009F
:1008B000877F8093E10082E08093180110921401F9
:1008C0008091E1008E7F8093E1008091E2008E7F35
:1008D0008093E2008091E20080618093E20042E038
:1008E00060E080E02BDE72D1FF91EF91BF91AF917C
:1008F0009F918F917F916F915F914F913F912F9138
:100900000F900FBE0F901F9018951F93CF93DF93FA
:10091000CDB7DEB7AA970FB6F894DEBF0FBECDBF36
:10092000E9E1F1E08091F100819321E0E132F20709
:10093000C9F75FDC8091E80083FF30C18091190125
:1009400090911A01953009F483C030F49130A9F1E7
:1009500068F0933091F122C1983009F4EFC09930DA
:1009600009F4FBC0963009F019C194C0803821F019
:10097000823809F013C108C08091150190911601C9
:10098000992389F082600FC080911D018F7087309C
:1009900008F004C18093E9008091EB0085FB882773
:1009A00080F91092E9009091E800977F9093E80019
:1009B0008093F1001092F100CCC0282F2D7F09F018
:1009C000EDC0882319F0823061F0E8C080911B01EE
:1009D000813009F0E3C0933009F080E08093160184
:1009E0002EC080911B0181112AC080911D018F7042
:1009F0002FEF280F263008F0D1C08093E900209116
:100A0000EB0020FF1CC0933021F48091EB0080624A
:100A100014C09091EB0090619093EB0021E030E0E6
:100A2000A90102C0440F551F8A95E2F74093EA00DE
:100A30001092EA008091EB0088608093EB001092A6
:100A4000E9008091E800877F8093E800E9DDA6C097
:100A50008111A4C010911B011F778091E300807861
:100A6000812B8093E3008091E800877F8093E800EA
:100A7000D7DD8091E80080FFFCCF8091E3008068A3
:100A80008093E300111102C082E001C083E08093F3
:100A9000180184C08058823008F080C080911B010A
:100AA00090911C018C3D53E0950771F583E08A839A
:100AB0008AE289834FB7F894DE01139620E03EE086
:100AC00051E2E32FF0E050935700E49120FF03C080
:100AD000E295EF703F5FEF708E2F90E0EA3010F0FC
:100AE000C79601C0C0968D939D932F5F243149F71F
:100AF0004FBF8091E800877F8093E8006AE270E052
:100B0000CE0101961CDC14C060911D0170911E0184
:100B1000AE014F5F5F4F88DBBC01892B09F43EC0FB
:100B20009091E800977F9093E80089819A81A5DCF5
:100B30008091E8008B778093E80030C0803871F5B1
:100B40008091E800877F8093E80080911401809372
:100B5000F1008091E8008E7777CF81111FC08091DE
:100B60001B0190911C0199270297C4F48091E80021
:100B7000877F8093E80080911B018093140150DDF2
:100B800080911401811106C08091E30087FD02C0AD
:100B900081E001C084E08093180122DB8091E800AD
:100BA00083FF0AC08091E800877F8093E8008091EE
:100BB000EB0080628093EB00AA960FB6F894DEBF3C
:100BC0000FBECDBFDF91CF911F9108950895CF93B0
:100BD00080911801882399F0C091E900CF7090911D
:100BE000EC00892F817090FD80E8C82B1092E900FD
:100BF0008091E80083FD89DECF70C093E900CF913A
:100C000008956F927F928F929F92AF92BF92CF92F0
:100C1000DF92EF92FF920F931F93CF93DF9300D059
:100C20001F92CDB7DEB77C01ADB6BEB68091E800AD
:100C300083FF03C1F701808190E020911D01309175
:100C40001E012817390709F0F8C080911A01833076
:100C500009F49AC030F4813071F0823009F4D1C0C7
:100C6000ECC08A3009F4B5C08B3009F49EC08930DD
:100C700009F0E3C04CC080911901813A09F0DDC050
:100C80008DB69EB61A82198280911B0110911C01AB
:100C90008B83F7018085482F50E08DB79EB7841B6A
:100CA000950B0FB6F8949EBF0FBE8DBFEDB7FEB784
:100CB00031966F0160E070E0CF01B8D14FEF410F86
:100CC0008E010F5F1F4F9601BE016D5F7F4FC70101
:100CD0009FDAF70186819781009721F0408550E0E7
:100CE000B6019BD11092E9008091E800877F809344
:100CF000E8008B8181118093F10069817A81C601BE
:100D00001EDB8091E8008B778093E80037C08091EC
:100D10001901813209F091C08DB69EB600911F0174
:100D20001091200170901B0160901C018DB79EB73F
:100D3000801B910B0FB6F8949EBF0FBE8DBFEDB711
:100D4000FEB731966F018091E800877F8093E800BD
:100D5000B801CF0152DB8091E8008E778093E800E4
:100D600021E0711001C020E030E0021B130B2C0DBC
:100D70003D1D4FEF460D672DC70155DA0FB6F894AC
:100D80009EBE0FBE8DBE59C080911901813A09F0F7
:100D900054C08091E800877F8093E8008091E8004C
:100DA00080FFFCCFF701818540C08091190181321D
:100DB00009F043C08091E800877F8093E80030DC31
:100DC00090911B0181E0911101C080E0F7018187C2
:100DD00034C080911901813281F58091E800877FCC
:100DE0008093E8001DDC80911B0190911C018827F5
:100DF00036E0969587953A95E1F7F70195878487D0
:100E00001CC080911901813AC1F48091E800877F6C
:100E10008093E8008091E80080FFFCCFF701848593
:100E2000958596958795969587958093F100809105
:100E3000E8008E778093E800F3DB0FB6F894BEBE2F
:100E40000FBEADBE0F900F900F90DF91CF911F910D
:100E50000F91FF90EF90DF90CF90BF90AF909F9059
:100E60008F907F906F900895FC01399627E0DF0105
:100E70001D922A95E9F721E0FC01218724EF31E05A
:100E80003587248723E0248361E001968CCB5F9231
:100E90006F927F928F929F92AF92BF92CF92DF928A
:100EA000EF92FF920F931F93CF93DF9300D01F9287
:100EB000CDB7DEB77C01ADB6BEB6809118018430E7
:100EC00009F086C08091E4009091E500F701228549
:100ED00033852817390709F47BC081818F7080938F
:100EE000E9008091E80085FF73C08DB69EB640850D
:100EF00050E08DB79EB7841B950B0FB6F8949EBF3C
:100F00000FBE8DBFEDB7FEB731966F011B821A82FF
:100F1000198260E070E0CF0189D08E010F5F1F4F12
:100F2000960140E0BE016D5F7F4FC70171D9582E19
:100F3000F70184859585892B29F011E086859785B1
:100F4000892B09F010E0F701668077806114710445
:100F500081F049815A81B301C60152D001E0892B49
:100F600009F400E0F701408550E0B601C30155D017
:100F700001C000E089819A81892BF1F0511004C0F1
:100F8000011102C010FF18C0F7018485958597876D
:100F9000868781818F708093E9008B818111809396
:100FA000F10069817A8140E050E0C6017ED98091EC
:100FB000E8008E778093E8008091E4009091E5004E
:100FC000F701938782870FB6F8949EBE0FBE8DBE41
:100FD0000FB6F894BEBE0FBEADBE0F900F900F902F
:100FE000DF91CF911F910F91FF90EF90DF90CF9005
:100FF000BF90AF909F908F907F906F905F9008957B
:10100000FB01DC0104C08D910190801921F4415055
:101010005040C8F7881B990B0895FB01DC0102C002
:1010200001900D9241505040D8F70895DC0101C065
:0E1030006D9341505040E0F70895F894FFCFC3
:10103E000081080000011001040000000000000003
:00000001FF
